:0A1E92000001020203030404050529
:071357004420C80000000063
:100F1200E4F567F566F565F564C203C200C202C274
:100F2200011210C97E187F008E0F8F107519187567
:100F32001A12750D18750E1C751518751658751B35
:100F420018751C71EE54E070030210567568007536
:100F520069808E6A8F6BC374AD9FFF74189ECF2415
:100F620002CF3400FEE48F638E62F561F560F55FB7
:100F7200F55EF55DF55CAF63AE62AD61AC60AB5F33
:100F8200AA5EA95DA85CC3120A5F5026E569255FC7
:100F9200F582E568355EF58374CDF0E55F2401F5F1
:100FA2005FE4355EF55EE4355DF55DE4355CF55C88
:100FB20080C4E4F55FF55EF55DF55CAF63AE62ADEE
:100FC20061AC60AB5FAA5EA95DA85CC3120A5F5008
:100FD20031AE5EAF5FE56B2FF582E56A3EF583E0E9
:100FE200FDE5692FF582E5683EF583EDF0EF24011A
:100FF200F55FE43EF55EE4355DF55DE4355CF55C98
:1010020080B985680F85691074002480FF741834D4
:10101200FFFEC3E51A9FF51AE5199EF519C3E512FD
:101022009FF512E5119EF511C3E5149FF514E51322
:101032009EF513C3E50E9FF50EE50D9EF50DC3E576
:10104200169FF516E5159EF515C3E51C9FF51CE5E3
:101052001B9EF51BD2E843D82090E668E04409F0D5
:1010620090E65CE0443DF0D2AFD288D28AC2A8C2F8
:10107200AA43E808D2FB90E680E020E105D20812FC
:101082001BAD90E680E054F7F0538EF8C2033001B6
:1010920005120B0AC201300329121EA85024C203F2
:1010A200121C8120001690E682E030E704E020E185
:1010B200EF90E682E030E604E020E0E4121BDC126E
:0710C2001EAA120D2E80C7CB
:100B0A0090E6B9E07003020BBB147003020C3824A0
:100B1A00FE7003020CBB24FB7003020BB5147003B6
:100B2A00020BAF14607314607624056003020D1A79
:100B3A00121EAC4003020D2690E6BBE024FE6022A2
:100B4A0014603324FD601114602224067048E50FF6
:100B5A0090E6B3F0E5108037E51990E6B3F0E51AB0
:100B6A00802DE51190E6B3F0E5128023E51390E6B7
:100B7A00B3F0E514801990E6BAE0FF121C08AA0641
:100B8A00A9077B01EA494B600DEE90E6B3F0EF90BE
:100B9A00E6B4F0020D26020D1F121E64020D261283
:100BAA0016F8020D26121E04020D26121E52020DFE
:100BBA0026121EAE4003020D2690E6B8E0247F609E
:100BCA001514601924027063A200E43325E0FFA221
:100BDA0002E4334F8041E490E740F0803F90E6BC66
:100BEA00E0547EFF7E00E0D394807C0040047D01C7
:100BFA0080027D00EC4EFEED4F2492F582741E3E7B
:100C0A00F583E493FF3395E0FEEF24A1FFEE34E68B
:100C1A008F82F583E0540190E740F0E4A3F090E678
:100C2A008AF090E68B7402F0020D26020D1F121E46
:100C3A00B04003020D2690E6B8E024FE60162402B6
:100C4A006003020D2690E6BAE0B40105C200020D67
:100C5A0026020D1F90E6BAE0705590E6BCE0547E7D
:100C6A00FF7E00E0D394807C0040047D0180027DF9
:100C7A0000EC4EFEED4F2492F582741E3EF583E49D
:100C8A0093FF3395E0FEEF24A1FFEE34E68F82F561
:100C9A0083E054FEF090E6BCE05480131313541F13
:100CAA00FFE0540F2F90E683F0E04420F0806D803F
:100CBA0064121EB2506690E6B8E024FE601924025F
:100CCA00705A90E6BAE0B40104D200804F90E6BAB6
:100CDA00E064026047803E90E6BCE0547EFF7E00FE
:100CEA00E0D394807C0040047D0180027D00EC4EBC
:100CFA00FEED4F2492F582741E3EF583E493FF3392
:100D0A0095E0FEEF24A1FFEE34E68F82F58380089A
:100D1A00120080500790E6A0E04401F090E6A0E0BF
:030D2A004480F012
:010D2D0022A3
:03005B000212216D
:0F122100C0E0C083C082C0D075D000C006C00737
:10123000AF91530780EF6480600302134A53917F9C
:10124000E55564017003021347E55464017048D307
:10125000E53A9464E5399400500302134790204323
:10126000E551F0A3E552F0D39464E5519400401E9B
:10127000D3E55294DCE55194005013E53A948AE5A5
:101280003994025009752C01755400752D0185396A
:1012900051853A52021341E55464027065C3E53A40
:1012A0009464E53994004048D3E53A9464E5399470
:1012B000004010D3E53A94DCE53994005005752CD4
:1012C000008027D3E53A94DCE5399400400FD3E55C
:1012D0003A9452E53994035004052C800DD3E53A35
:1012E0009452E53994034008052C753900753A008D
:1012F000E52C652F7002E52E704DF554F539F53A61
:101300008045E554B40540D3E53A9401E5399400AD
:101310004035E53825E0FFE53733FE74412FF5828F
:1013200074203EF583E539F0A3E53AF00538E53859
:1013300070020537052CE52CB41406755400752C85
:0A13400000753900753A007555007C
:0D134A00D007D006D0D0D082D083D0E032C2
:030003000219528D
:10195200C0E0C0F0C083C082C0D075D000C000C05B
:1019620004C005C006C00790E6017443F0E5537059
:10197200600541E541B40903753B019020C8E0FCD4
:10198200A3E0FDA3E0FEA3E02401FFE43EFEE43D6C
:10199200FDE43CFC9020C8120A8390F00074AAF087
:1019A200A37411F0A374CCF0A374EEF090E690E46B
:1019B200F090E6917405F0300419AF3FAE3EAD3DB4
:1019C200AC3C8F0C8E0B8D0A8C0975080FD20780E8
:1019D200021553A283B39283D007D006D005D00458
:0D19E200D000D0D0D082D083D0F0D0E03241
:03000B000219EFE8
:1019EF00C0E0C0F0C083C082C0D075D000C000C0BE
:1019FF0001C002C003C004C005C006C00785278C04
:101A0F0085288AE5086016D2831508E508704C9082
:101A1F00E600E054FDF0000000C283803E30073B3B
:101A2F00AF0CAE0BAD0AAC09EF24FFF50CEE34FF93
:101A3F00F50BED34FFF50AEC34FFF509E4FFFEFD7D
:101A4F00FCAB0CAA0BA90AA809C3120A5F700CC23F
:101A5F000790E600E04402F0000000D007D006D067
:101A6F0005D004D003D002D001D000D0D0D082D086
:061A7F0083D0F0D0E0323C
:03003300021EA406
:041EA40053D8EF32EE
:10135E00608020410000000000000000000000003E
:10136E00000000000000000000000000000000006F
:10137E00000000000000000000000000000000005F
:10138E00000000000000000000000000000000004F
:10139E00000000000000000000000000000000003F
:1013AE00000000000000000000000000000000002F
:1013BE00000000000000000000000000000000001F
:1013CE00000000000000000000000000000000000F
:1013DE0000000000023700000127D101284A014712
:1013EE0000043C00000000C107C104012B000448AA
:1013FE00000000000442000000004120C700412010
:10140E00C300422002000042200400004120C4001C
:10141E0042201900004220C100004220000000427C
:10142E00201D000042201B007E4220C50000014608
:10143E00BA0154FF022EFFFF012C300239000002C8
:10144E00510000045700000000024E00000423006B
:10145E0000000004330000C35002290064014D0057
:10146E00012D00015000014100013B00023000003F
:101DC20085278C85288AE58954F04401F589438E5C
:061DD20008D28CD2A92208
:061D7900C2817F647E00C0
:101D7F00EF25E0FFEE33FEEF4E6007EF1F70F81E0A
:031D8F0080F522BA
:101D0700AD07AC06ED4C60147F957E00121D7F0079
:0D1D17000000000000ED1D70EB1C80E822B4
:101CC90090E6187408F000000090E619F000000092
:0F1CD90090E61AF000000090E61BF000000022D9
:101CE80090E6187409F000000090E619F000000072
:0F1CF80090E61AF000000090E61BF000000022BA
:0E1E760090201FEDF07D1F7B017A00021D5DA4
:1010C90090E6007412F090E60B7403F000000090B3
:1010D900E6047480F00000007402F000000074045B
:1010E900F00000007406F00000007408F000000031
:1010F900E4F000000000000090E61274E8F000003F
:1011090000E490E613F000000090E614F0000000FF
:1011190090E615F000000090E6187408F000000051
:1011290090E619F000000090E61AF000000090E641
:101139001BF000000090E6097404F000000090E63E
:1011490070E04401F0000000E490E672F000000055
:1011590090E6207402F0000000E490E621F000001F
:101169000090E602F000000090E603F090E60174BA
:1011790043F000000090E61174A0F000000090E632
:101189005EE04404F000000090E68F7440F0000037
:101199000090E61074A0F000000090E65EE04408BC
:1011A900F0000000E490E68DF043AF01D20043B2B5
:1011B9000843B20275B6FF75B1F075B4FF121E9CF3
:1011C900121D79D281121DC275752075763F7B0279
:1011D9007D107FA0121C5C90203FE0F556A3E0F53E
:1011E90032E55664066005E556B40705754620D212
:1011F90006E4F553D283755501F539F53A53A0F054
:1012090043A04043E80875540190201FF07A207BE1
:081219001F7D017F48021D5DED
:0E1E8400EF2401FBE43EFA7D027F48021D417F
:101E1900851E82851D83EFF0AB1EAA1D7D017F21E2
:031E2900021D5D3A
:101E2C00857F82857E83EFF0AB7FAA7E7D017F2745
:031E3C00021D5D27
:1006BE00756C7FE4F56DF56E7EE77FC0121E847853
:1006CE001F7C207D017B017AE779C07E007F0412BA
:1006DE0009B49020C4E0702CE547D39400401F432A
:1006EE00A0807540FFE54713FFC3747F9FF56CE54F
:1006FE00476401600302088C756C7F02088C53A05E
:10070E007F02088C43A080902020E0FEA3E07C00B6
:10071E002400FFEC3E902000F0FCA3EFF0FD9020B3
:10072E0003E0FE902005E02400FF902004E03EFE52
:10073E0090201DF0A3EFF0D3ED9FEC9E405E902035
:10074E00C77401F090201DE0FEA3E0FF902001E0B1
:10075E009FFF902000E09E9020C1F0A3EFF090202C
:10076E00C1E0C4F854F0C868F56DA3E0C4540F4856
:10077E00F56E90201BE0FEA3E0FFD3956EEE956D17
:10078E004010EF956EFFEE956D90201BF0A3EFF0ED
:10079E00805B90201BE4F0A304F08051E49020C70E
:1007AE00F0902000E0FEA3E0FFC390201EE09FFF2C
:1007BE0090201DE09E9020C1F0A3EFF09020C1E0AC
:1007CE00C4F854F0C868FEA3E0C4540F48FF90204C
:1007DE001CE02FF090201BE03EF0D3A3E0947E901F
:1007EE00201BE094004006E4F0A3747EF09020C33A
:1007FE00E06032902019E0FEA3E07805CEC313CE60
:10080E0013D8F9FF90201CE02FF090201BE03EF053
:10081E00D3A3E0947E90201BE094004044E4F0A328
:10082E00747EF0803C902019E0FEA3E07805CEC3E4
:10083E0013CE13D8F9F56E8E6D90201BE0FEA3E05B
:10084E00FFD3956EEE956D4010EF956EFFEE956DA4
:10085E0090201BF0A3EFF0800890201BE4F0A3047F
:10086E00F09020C1E0FFA3E0902019CFF0A3EFF0AD
:10087E009020C7E09020C3F090201CE0F56C9020F3
:10088E00C5E07004A3E0640A601AE56CC3943F509F
:10089E0003756C3F9020C6E004F070119020C5E007
:1008AE0004F080099020C5E4F0A3740AF090201F94
:1008BE007402F0A37480F07A207B1F7D027F2812D1
:1008CE001D5DE490201FF0A3E56CF07A207B1F7D68
:0608DE00027F28021D5DEF
:100D2E00E55A2401F55AE43559F559E43558F55884
:100D3E00E43557F557054FE54F7002054EAF36AE09
:100D4E0035AD34AC33AB5AAA59A958A857C3120AB9
:100D5E005F700C1206BEE4F55AF559F558F557902A
:100D6E00E7C8E554F0A3E52CF0A3E53BF0E54F65AD
:100D7E002A7004E54E65297028E554601624FE603D
:100D8E000D24FD600924047013121E3F800E1217ED
:100D9E00EF800953B10F53A0BF43A00FE4F54EF5FA
:100DAE004FE52B64017036FFFEFDE548FC78181206
:100DBE000A7090E7C4EFF0E4FFFEE549FDE4FC782D
:100DCE0010120A70A3EFF0E4FFE54AFEE4FDFC7892
:100DDE0008120A70A3EFF0E54BFFA3EFF0E52B64CA
:100DEE00026003020F11FFFEFDE548FC7818120A9F
:100DFE007090E7C4EFF0E4FFFEE549FDE4FC7810E7
:100E0E00120A70A3EFF0E4FFE54AFEE4FDFC780859
:100E1E00120A70A3EFF0E54BFFA3EFF0C283208020
:100E2E00FD7F057E0012167B90E600E054FDF0E497
:100E3E00F526F525F524F523854B45854A44854948
:100E4E0043854842E47F64FEFDFCAB45AA44A943BA
:100E5E00A842D3120A5F5003020EF67F647E001280
:100E6E00167BE545249CF545E54434FFF544E54302
:100E7E0034FFF543E54234FFF542E4FFFEFDE54263
:100E8E00FC7818120A7090E7C4EFF0E4FFFEE54319
:100E9E00FDE4FC7810120A70A3EFF0E4FFE544FEC7
:100EAE00E4FDFC7808120A70A3EFF0E545FFA3EF0E
:100EBE00F0E47F0AFEFDFCAB26AA25A924A823C3D5
:100ECE00120A5F700BF526F525F524F5231206BEE2
:100EDE00E5262401F526E43525F525E43524F5240B
:100EEE00E43523F523020E52AE44AF4512167B9025
:100EFE00E6017440F090E600E04402F0D2A8C2830E
:040F0E00E4F52B22B9
:021EA800D32243
:021EAA00D32241
:021EAC00D3223F
:101E040090E680E030E704D2058002C20590E6BA8D
:051E1400E0F54CD322B3
:101E520090E740E54CF0E490E68AF090E68B04F0DF
:021E6200D32289
:0816F80090E6BAE0F522D322CE
:101E640090E740E522F0E490E68AF090E68B04F0F7
:021E7400D32277
:021EAE00D3223D
:021EB000D3223B
:021EB200D32239
:10008000E4F570F57190E6B9E0120A8F00CFB30085
:10009000F3B70139B8019AB901B8BB0271BD02B317
:1000A000BF02C2C002F5C104CCC2050FC5052AC6F5
:1000B0000551C80578C905FBCA0628CB067BCD06C5
:1000C000AACF0350D004B4D10442D2000006BAC271
:1000D000A890E6017440F000000090E6047480F0FF
:1000E0000000007402F0000000E4F0000000D2A85C
:1000F00002069A90E6BDE0FE90E6BCE07C0024009B
:10010000F56DEC3EF56C200617AD6D90E6BEE0FB9C
:100110007EE77575E7757640AF46121C5C020617E0
:1001200090E6BEE0FB7EE77576E7757740AD6DAC97
:100130006CAF46121C34020617E490E68AF090E693
:100140008BF090E6A0E020E1F9E4F56EF56FAF6F7B
:1001500074402FF582E434E7F583E0FE74062FF552
:1001600082E43420F583EEF0056FE56F7002056ED2
:100170006413456E70D8902006E070031200009062
:100180002006E0B40103120000902006E064026043
:10019000030206BC1200000206BCE490E68AF0905E
:1001A000E68BF090E6A0E020E1F9E546C313FF7A84
:1001B000E77B407D03020676E490E68AF090E68BCA
:1001C000F090E6A0E020E1F920063B781F7C207D3E
:1001D000017B017AE679BC7E007F011209B490E6CA
:1001E000BEE0FF7E0078207C207D017B017AE779EC
:1001F000401209B4E546C313FF90E6BEE004FD7A61
:10020000207B1F02067690E6BDE0FE90E6BCE07C17
:10021000002400FFEC3EFEBE3E08BFE405E4F53BD3
:10022000F541781F7C207D017B017AE679BD7E0057
:100230007F011209B478207C207D017B017AE67968
:10024000BC7E007F011209B490E6BEE0FF7E00781C
:10025000217C207D017B017AE779401209B4E546D3
:10026000C313FF90E6BEE02402FD7A207B1F020646
:1002700076E490E68AF090E68BF090E6A0E020E14C
:10028000F990E740E0FCA3E0FDA3E0FEA3E0F53F2A
:100290008E3E8D3D8C3CE4FFFEFDFCAB3FAA3EA9AB
:1002A0003DA83CC3120A5F7005C204020333D204A6
:1002B000020333E4F508C20790E600E04402F000D0
:1002C000000090E6BAE030E01190E6BCE05490C443
:1002D000540FFFE5B154F64FF5B190E6BAE030E1C6
:1002E0001190E6BCE05460C4540FFFE5B154F94FDF
:1002F000F5B10206AFE490E68AF090E68BF090E666
:10030000A0E020E1F990E740E0FCA3E0FDA3E0FEDF
:10031000A3E0F53F8E3E8D3D8C3CE4FFFEFDFCAB43
:100320003FAA3EA93DA83CC3120A5F7004C20480E4
:1003300002D204E4F508C20775530190E600E044D8
:1003400002F0000000E490E68AF00000000206B42B
:10035000E490E68AF090E68BF090E6A0E020E1F9E8
:1003600090E68BE0756E00F56FC29890E740E0C3B1
:1003700094304006E0D39438400A90E740E0F460BF
:1003800003020424E554600302042490E740E0F4EF
:10039000600AE0B43017E52C6401601153A0F0430B
:1003A000A040755501755401E4F54D807790E74004
:1003B000E0C39431406EE0D394385068E024D1F526
:1003C0002FE434FFF52EE52C652F7002E52E6054E6
:1003D00053A0F043A040E0B40A06752E00752F61CB
:1003E00090E740E0B40B06752E00752F6290E74051
:1003F000E0B40C06752E00752F6390E740E0B40D55
:1004000006752E00752F6490E740E0B40E06752E39
:1004100000752F6590E740E0B40F06752E00752F2C
:100420006675540290E740E0642060030206BCE574
:100430005460030206BC53A0F043A040755405026B
:1004400006BCC3E5719414E570648094805052AE8C
:1004500070AF717C007D02120A29EF25E0FDEE33BA
:10046000FC74412DF58274203CF583E0FFAE71747D
:10047000402EF582E434E7F583EFF074412DF582E8
:1004800074203CF583A3E0FF74412EF582E434E749
:10049000F583EFF074022571F571E43570F5708025
:1004A000A1000000E490E68AF000000090E68B7462
:1004B000280206A490E740E52DF0000000E490E655
:1004C0008AF000000090E68B040206A490E74074D6
:1004D00008F0A3740CF0E4A3F0A3F0A3F0A2063399
:1004E000A3F0A3E532F0A3E546F0A3E556F030050E
:1004F00005E4A3F0800690E74974FFF0000000E4F3
:1005000090E68AF000000090E68B740A0206A47E52
:10051000E77F40121E84000000E490E68AF00000AD
:100520000090E68B7404F00206BCE490E68AF0903A
:10053000E68BF090E6A0E020E1F990E740E0FD7F57
:100540004E121E7690E741E0FD7F42121E760206B3
:10055000BCE490E68AF090E68BF090E6A0E020E123
:10056000F990E740E014600C14600B240260030271
:1005700006BC80258041805FE490E68AF090E68B9F
:10058000F090E6A0E020E1F990E740E01460281444
:100590006045240260030206BC7527F47528539059
:1005A000E6007402F0E47536507535C3F534F53362
:1005B000F529752A19803E7527E87528A590E6006B
:1005C000740AF07536A0753586753401753300757B
:1005D0002900752A32801E7527D175284A90E600B9
:1005E0007412F075364075350D753403753300752A
:1005F0002900752A64121E9C0206BC90E6BCE075B8
:100600006C00F56DFD90E6BEE0FB7EE77575E77565
:1006100076407FA0121C5CE490E68AF00000009017
:10062000E6BEE090E68B807CE490E68AF090E68B74
:10063000F090E6A0E020E1F990E6BCE0D39407401A
:100640007B781F7C207D017B017AE679BC7E007F70
:10065000011209B490E6BEE0FF7E0078207C207D88
:10066000017B017AE779401209B490E6BEE004FD0F
:100670007A207B1F7F50121D5D8041E490E68AF056
:1006800090E68BF090E6A0E020E1F990E740E07082
:1006900005121CC98003121CE8E490E68AF00000F1
:1006A0000090E68BF00000008012121D79D281E4E8
:0D06B00090E68AF090E68BF08002D322C322
:0106BD00221A
:101D9200C0E0C083C082D2015391EF90E65D74012E
:081DA200F0D082D083D0E032C2
:101DD800C0E0C083C0825391EF90E65D7404F0D0F8
:061DE80082D083D0E0323E
:101DEE00C0E0C083C0825391EF90E65D7402F0D0E4
:061DFE0082D083D0E03228
:1016C100C0E0C083C08290E680E030E70E850D1156
:1016D100850E12851513851614800C851511851636
:1016E10012850D13850E145391EF90E65D7410F081
:0716F100D082D083D0E0326B
:101DAA00C0E0C083C082D2035391EF90E65D74080D
:081DBA00F0D082D083D0E032AA
:1017B800C0E0C083C08290E680E030E70E850D115E
:1017C800850E12851513851614800C85151185163E
:1017D80012850D13850E145391EF90E65D7420F079
:0717E800D082D083D0E03273
:0117FF0032B7
:011EB40032FB
:011EB50032FA
:011EB60032F9
:101CA600C0E0C083C08200000090E68F7440F00060
:101CB60000005391EF90E65FE04404F0D082D083B9
:031CC600D0E03239
:10158700C0E0C083C082C0D075D000C004C005C011
:0315970006C00784
:10159A0090E6A1E020E1F990E780E014601D146074
:1015AA002E24F26051146065147003021647241346
:1015BA00600614600302165802164C90E782E0F5A2
:1015CA004090E781E0F5479020C4E4F0A3802290A0
:1015DA00E782E0FF902002E4F0A3EFF090E781E0D9
:1015EA00FF902004E4F0A3EFF09020C47401F0A36C
:1015FA00E4F0A3F0805890E781E0FCA3E0FDA3E0CB
:10160A00FEA3E0F54B8E4A8D498C488041752B012B
:10161A00C2A8D28390E600E04402F000000090E6FF
:10162A00017440F000000090E6047480F0000000AD
:10163A007402F0000000E4F00000008011752B0233
:10164A00800C7545647544007543007542000000BE
:10165A000090E68DE4F05391EF90E65FE04408F0E5
:10166A00D007D006D005D004D0D0D082D083D0E025
:01167A00323D
:011EB70032F8
:011EB80032F7
:011EB90032F6
:011EBA0032F5
:011EBB0032F4
:011EBC0032F3
:011EBD0032F2
:011EBE0032F1
:011EBF0032F0
:011EC00032EF
:011EC10032EE
:011EC20032ED
:011EC30032EC
:011EC40032EB
:011EC50032EA
:011EC60032E9
:011EC70032E8
:011EC80032E7
:011EC90032E6
:011ECA0032E5
:011ECB0032E4
:011ECC0032E3
:011ECD0032E2
:011ECE0032E1
:011ECF0032E0
:011ED00032DF
:011ED10032DE
:011ED20032DD
:011ED30032DC
:011ED40032DB
:041C5C008F728B7484
:101C60009020CCEDF0E572C313FF7A207BCC7D0190
:101C7000121D5DE572C313FFAB76AA75AD74021D2C
:011C80004122
:041C34008F728B75AB
:101C3800EC9020CCF0EDA3F0E572C313FF7A207B83
:101C4800CC7D02121D5DE572C313FFAB77AA76AD9A
:041C580075021D41B3
:101D2400A907EC90201FF0EDA3F0EAA3F0EBA3F0D9
:0D1D3400E9C313FF7A207B1F7D04021D5DB3
:1018AF000531E53170020530640845307004F530BC
:1018BF00F531E5314530700843B12053B1EF806900
:1018CF00E53164014530700543B120800BE531648B
:1018DF00024530700B53B1DF53B1EF43B140805F1E
:1018EF00E53164034530700B53B1DF53B1EF43B1B2
:1018FF00408024E53164044530700B53B1DF53B1A0
:10190F00EF53B1BF8011E53164054530700D53B110
:10191F00DF43B11053B1BF43B18022E531640645B7
:10192F0030700B53B1DF43B11053B1BF8011E531AC
:10193F0064074530700C43B12043B11053B1BF530E
:03194F00B17F2243
:101E3F00E4F52DE554600B1218AF053AE53A700240
:031E4F0005392230
:1017EF00E554600B053AE53A700205391218AF223D
:101800001201000200000040181631090000010218
:1018100000010A06000200000040010009023C002D
:1018200001010080FA0904000006FF00000007051E
:101830008202000200070501020002000705020201
:1018400000020007050602000200070581020002EF
:10185000000705860200020009021900010100804C
:10186000FA0904000001FF000000070582024000A1
:10187000000403090414035100480043002D0043F1
:101880000043004400200020002403510048005978
:10189000002D006D0069006E006900430061006D5D
:0F18A00000350020002000200020002000000064
:101BDC0090E682E030E004E020E60B90E682E03014
:101BEC00E119E030E71590E680E04401F07F147EC7
:0C1BFC000012167B90E680E054FEF02200
:101C810090E682E044C0F090E681F04387010000D5
:041C9100000000222D
:101BAD0030080990E680E0440AF0800790E680E076
:101BBD004408F07FDC7E0512167B90E65D74FFF025
:0F1BCD0090E65FF05391EF90E680E054F7F0223E
:10167B008E6C8F6D90E600E054187012E56D2401AE
:10168B00FFE4356CC313F56CEF13F56D801590E625
:10169B0000E05418FFBF100BE56D25E0F56DE56C10
:1016AB0033F56CE56D156DAE6C7002156C4E600507
:0616BB00121C9580EE22D6
:081E9C00E4F57DD2E9D2AF228A
:101B110090E678E020E6F9C2E990E678E04480F0CA
:101B2100EF25E090E679F090E678E030E0F990E694
:101B310078E04440F090E678E020E6F990E678E03D
:061B410030E1D6D2E922DA
:101B7B00A90790E678E020E6F9E57D702390E678FA
:101B8B00E04480F0E925E090E679F08D78AF03A989
:101B9B00077579018A7A897BE4F57C757D01D322FF
:021BAB00C32253
:101B4700A90790E678E020E6F9E57D702590E6782C
:101B5700E04480F0E925E0440190E679F08D78AF24
:101B670003A9077579018A7A897BE4F57C757D037A
:041B7700D322C32290
:03004B0002147F1D
:10147F00C0E0C083C082C085C084C086758600C0AE
:10148F00D075D000C000C001C002C003C006C007A5
:10149F0090E678E030E206757D0602156990E678F1
:1014AF00E020E10CE57D64026006757D0702156999
:1014BF00E57D24FE605F14603624FE700302155A2A
:1014CF0024FC700302156624086003021569AB79CA
:1014DF00AA7AA97BAF7C057C8F827583001209DA0B
:1014EF0090E679F0E57C65787070757D05806B907E
:1014FF00E679E0AB79AA7AA97BAE7C8E8275830000
:10150F00120A07757D02E5786401704E90E678E067
:10151F004420F08045E57824FEB57C0790E678E01E
:10152F004420F0E57814B57C0A90E678E04440F06A
:10153F00757D0090E679E0AB79AA7AA97BAE7C8EB7
:10154F0082758300120A07057C800F90E678E044CD
:10155F0040F0757D008003757D005391DFD007D07B
:10156F0006D003D002D001D000D0D0D086D084D006
:08157F0085D082D083D0E03258
:021C0800A9072A
:101C0A00AE1BAF1C8F828E83A3E064037017AD01F5
:101C1A0019ED7001228F828E83E07C002FFDEC3E4D
:091C2A00FEAF0580DF7E007F00A3
:011C3300228E
:101D4100121B47E57D24FA600E146006240770F328
:0C1D5100D322E4F57DD322E4F57DD322FB
:101D5D00121B7BE57D24FA600E146006240770F3D8
:0C1D6D00D322E4F57DD322E4F57DD322DF
:101C95007400F58690FDA57C05A3E582458370F962
:011CA500221C
:03004300021700A1
:0300530002170091
:10170000021D9200021DEE00021DD800021DAA005B
:101710000216C1000217B8000217FF00021EB40033
:10172000021EB500021EB600021CA60002158700AC
:10173000021EB700021EB800021EB900021EBA0047
:10174000021EBB00021EB400021EBC00021EBD0031
:10175000021EBE00021EBF00021EC000021EC1000B
:10176000021EC200021EB400021EB400021EB4001B
:10177000021EC300021EC400021EC500021EC600D7
:10178000021EC700021EC800021EC900021ECA00B7
:10179000021ECB00021ECC00021ECD00021ECE0097
:1017A000021ECF00021ED000021ED100021ED20077
:0817B000021ED300021ED4004A
:03000000021A855C
:0C1A8500787FE4F6D8FD75817F021ACC52
:1008E400E709F608DFFA8046E709F208DFFA803EF6
:1008F40088828C83E709F0A3DFFA8032E309F608E3
:10090400DFFA8078E309F208DFFA807088828C834A
:10091400E309F0A3DFFA806489828A83E0A3F608FE
:10092400DFFA805889828A83E0A3F208DFFA804CD8
:1009340080D280FA80C680D4806980F280338010AF
:1009440080A680EA809A80A880DA80E280CA803318
:1009540089828A83ECFAE493A3C8C582C8CCC58390
:10096400CCF0A3C8C582C8CCC583CCDFE9DEE78060
:100974000D89828A83E493A3F608DFF9ECFAA9F0DF
:10098400EDFB2289828A83ECFAE0A3C8C582C8CC35
:10099400C583CCF0A3C8C582C8CCC583CCDFEADE4E
:1009A400E880DB89828A83E493A3F208DFF980CCB0
:1009B40088F0EF60010E4E60C388F0ED2402B404A9
:1009C4000050B9F582EB2402B4040050AF23234550
:0609D40082239009347338
:1009DA00BB010CE58229F582E5833AF583E02250D2
:1009EA0006E92582F8E622BBFE06E92582F8E2221C
:0D09FA00E58229F582E5833AF583E4932236
:100A0700F8BB010DE58229F582E5833AF583E8F025
:100A1700225006E92582C8F622BBFE05E92582C8D1
:020A2700F222B9
:100A2900C2D5EC30E709B2D5E4C39DFDE49CFCEEE8
:100A390030E715B2D5E4C39FFFE49EFE120AB5C3A1
:100A4900E49DFDE49CFC8003120AB530D507C3E49C
:060A59009FFFE49EFE2257
:100A5F00EB9FF5F0EA9E42F0E99D42F0E89C45F0ED
:010A6F002264
:100A7000E8600FECC313FCED13FDEE13FEEF13FF64
:030A8000D8F12288
:0C0A8300ECF0A3EDF0A3EEF0A3EFF022E6
:100A8F00D083D082F8E4937012740193700DA3A3F6
:100A9F0093F8740193F5828883E47374029368600A
:060AAF00EFA3A3A380DF0A
:101A9100020F12E493A3F8E493A34003F68001F24A
:101AA10008DFF48029E493A3F85407240CC8C33356
:101AB100C4540F4420C8834004F456800146F6DF25
:101AC100E4800B0102040810204080901357E47E4B
:101AD100019360BCA3FF543F30E509541FFEE4931A
:101AE100A360010ECF54C025E060A840B8E493A3E1
:101AF100FAE493A3F8E493A3C8C582C8CAC583CA0C
:101B0100F0A3C8C582C8CAC583CADFE9DEE780BEC3
:01147E00006D
:100AB500BC000BBE0029EF8DF084FFADF022E4CC25
:100AC500F875F008EF2FFFEE33FEEC33FCEE9DECEE
:100AD500984005FCEE9DFE0FD5F0E9E4CEFD22ED34
:100AE500F8F5F0EE8420D21CFEADF075F008EF2F7E
:100AF500FFED33FD4007985006D5F0F222C398FD6F
:050B05000FD5F0EA220B
:00000001FF
